:020000040000FA
:06000000FA6A18EF00F09F
:020006000000F8
:0800080080AA11EF00F0825004
:10001000E96EEF508A6E936A00000000931E16EF9F
:1000200000F08250E96E8150EF6EB888F0921000B7
:10003000700ED36E060ED26EDF0E9B6ED190100E38
:10004000776E786AFF0E926E7E6A7F6AFF0E936EFD
:10005000FF0E946EEA6AE26AD09EF198F088F29CF4
:1000600080A630EF00F080A846EF00F0FF0EE16EB2
:10007000E150A96EA69EA69CA680A850E76E010E30
:10008000E15ED8B038EF00F04FEF00F0FF0EE16E08
:10009000000EE76E010EE15ED8B048EF00F0F28E80
:1000A000B898B8A851EF00F080B654EF00F0F29E77
:1000B0009B6AD36AE26AFF0EE16EE1CFA9FFE750C7
:1000C000A86EA69EA69CA684550EA76EAA0EA76E25
:1000D000A682A6B269EF00F0A694010EE15ED8B048
:0E00E0005DEF00F080A672EF00F018EF00F068
:020000040030CA
:0100010028D6
:0100020018E5
:010003001EDE
:0100050008F2
:010006008079
:0100080003F4
:01000900C036
:01000A0003F2
:01000B00E014
:01000C0003F0
:01000D0040B2
:0200000400F00A
:1000000000000000000000000000000000000000F0
:1000100000000000000000000000000000000000E0
:1000200000000000000000000000000000000000D0
:1000300000000000000000000000000000000000C0
:1000400000000000000000000000000000000000B0
:1000500000000000000000000000000000000000A0
:100060000000000000000000000000000000000090
:100070000000000000000000000000000000000080
:100080000000000000000000000000000000000070
:100090000000000000000000000000000000000060
:1000A0000000000000000000000000000000000050
:1000B0000000000000000000000000000000000040
:1000C0000000000000000000000000000000000030
:1000D0000000000000000000000000000000000020
:1000E0000000000000000000000000000000000010
:1000F0000000000000000000000000000000000000
:00000001FF
